:0400000080EF01F09C
:100008003582FACF13F0FBCF14F0E9CF15F0EACF21
:1000180016F0E1CF17F0E2CF18F0D9CF19F0DACF08
:100028001AF0F3CF1BF0F4CF1CF0F6CF1DF0F7CF8A
:100038001EF0F8CF1FF0F5CF20F035C021F036C004
:1000480022F037C023F038C024F09EA22FD180CFF1
:1000580025F081CF26F0070E296E2950040D620E77
:10006800F324D96E000EF420DA6EDECF01F0DECF75
:1000780002F0DECF03F0DECF04F0D8900134056E35
:100088000234066E0334076E0434086E29C009F082
:1000980025C00AF0092A02D0D8900A32092EFCD7C6
:1000A800010E0A160A5005100B6E06500C6E07500A
:1000B8000D6E08500E6E2950040D620EF324D96E91
:1000C800000EF420DA6E0BC0DEFF0CC0DEFF0DC0A0
:1000D800DEFF0EC0DEFF2950016E026AD89001369D
:1000E8000236D89001360236200E0126000E022272
:1000F800620E0124D96E000E0220DA6EDECF03F004
:10010800DECF04F0DECF05F0DECF06F0D890033462
:10011800076E0434086E0534096E06340A6E29C069
:100128000BF026C00CF00B2A02D0D8900C320B2E04
:10013800FCD7010E0C160C5007100D6E08500E6EF1
:1001480009500F6E0A50106E2950116E126AD8901D
:1001580011361236D89011361236200E1126000E9E
:100168001222620E1124D96E000E1220DA6E0DC012
:10017800DEFF0EC0DEFF0FC0DEFF10C0DEFF000E88
:10018800276E2950040D620EF324D96E000EF42058
:10019800DA6EDE50DE10DE10DE10D8B41CD0295026
:1001A800040D620EF324D96E000EF420DA6E000EF0
:1001B800DE14016EFF0EDE14026EFF0EDE14036EF7
:1001C800FF0EDE14046E0150021003100410D8A4B0
:1001D80002D0010E276E29C001F02750026E036A73
:1001E800012A03D0D89002360336012EFBD70250DD
:1001F8000001601303506113000E286E2950016E30
:10020800026AD89001360236D89001360236200E9E
:100218000126000E0222620E0124D96E000E022071
:10022800DA6EDE50DE10DE10DE10D8B427D029508A
:10023800016E026AD89001360236D890013602362D
:10024800200E0126000E0222620E0124D96E000E35
:100258000220DA6E000EDE14036EFF0EDE14046E4A
:10026800FF0EDE14056EFF0EDE14066E035004103A
:1002780005100610D8A402D0010E286E29C001F07E
:10028800080E01262850026E036A012A03D0D8906E
:1002980002360336012EFBD70250000160130350CB
:1002A800611329062928D8A4D8D69E9224C038F0EC
:1002B80023C037F022C036F021C035F020C0F5FF4A
:1002C8001FC0F8FF1EC0F7FF1DC0F6FF1CC0F4FFDB
:1002D8001BC0F3FF1AC0DAFF19C0D9FF18C0E2FF2C
:1002E80017C0E1FF16C0EAFF15C0E9FF14C0FBFF05
:0C02F80013C0FAFF359211009CEF04F0D7
:100600000024002600280029002B002D002F003098
:1006100000320034003500370039003E003C003B1A
:100620000040004100430045004700001CEC04F07E
:10063000620E2A6E000E2B6E000E2D6E000E2C6EBA
:10064000000E2F6E400E2E6E45EC04F0F28E00016F
:10065000A751F00B0C09A76FA799A79BA79DA79F70
:10066000090EAA6F000EA96F010EA86FB00E2F6EB3
:10067000000E306E000E326E000E316E010EF66E00
:10068000060EF76E0800F5CF33F07F0E346EEBECFC
:1006900003F0290E0001A36F960EA26F7F0EE82EC5
:1006A000FED7A22FFCD7A32FFAD7A70E2B6E000ED2
:1006B0002C6EB1EC03F0000E0001AF6F000EAE6FB8
:1006C000AF51F9E1100EAE5DD8B0F5D7AEC0A2F0D3
:1006D000010EA36F000EA46FA22B03D0D890A337F6
:1006E000A437A22FFBD700016051A3176151A417B3
:1006F000A351A411D8B432D0D890AE35F66EAF3530
:10070000F76E010EF626060EF7220800F5CFB3F0BD
:10071000B00E2B6E000E2C6EB1EC03F0D00E00016B
:10072000A26FC90EE82EFED7A22FFCD700D0AEC014
:10073000A2F0010E0001A36F000EA46FA22B03D044
:10074000D890A337A437A22FFBD70001A31DA56F14
:10075000A41DA66FA5516017A6516117AE4BAF2B14
:10076000AFD72B502C10D8B4120020EE01F02B5034
:10077000D9262C50DA22DECF2FF0DDCF30F0030E59
:100780002B24316E000E2C20326E2BC0D9FF2CC0D2
:10079000DAFFDF380F0B2D6E2BC0D9FF2CC0DAFF2C
:1007A000DF500F0B2E6E2E38F00B2D10A9EC04F03D
:1007B00009D031C0D9FF32C0DAFFDF50A9EC04F014
:1007C000314A322A2F06D8A030062F28F2E13028ED
:1007D000D8B41200EED72F503010D8B412002FC06A
:1007E0002AF030C02BF0090E2C6E6EEC04F02FC0F6
:1007F0002AF030C02BF031C02CF032C02DF05BEC71
:1008000004F020EE03F02F50D9263050DA2233C006
:10081000DFFF20EE04F02F50D9263050DA2234C00A
:10082000DFFF20EE01F02F50D9263050DA22020EE1
:10083000DE6E000EDD6E1200F29E9B8C9B809B8212
:100840009B849B869B889B9AD388D38AD38CFC0EEF
:10085000D316000E0F01386F000E396F000E3A6F7D
:10086000000E3B6F92689368800EBB6EBA50870B88
:100870000809BA6E030EBA12BA849D829E92F28C57
:100880008EEC04F080EC04F012002AC030F02BC093
:1008900031F008D030C0D9FF31C0DAFF2CC0DFFF03
:1008A000304A312A2E06D8A02F062E28F3E12F2811
:1008B000D8B41200EFD72A502B10D8B412002CC095
:1008C0002EF00F0E2E162AC0D9FF2BC0DAFF2E3ABB
:1008D000DF502E180F0B2E18DF6E12002A502B102F
:1008E000D8B412002CC02DF00F0E2D162AC0D9FF3F
:1008F0002BC0DAFFDF502D18F00B2D18DF6E120021
:100900007298729C718E1F0E756E000E766E7294C8
:100910007096958E958C7188728A1200AC98AC9CFA
:10092000AB8E1F0EAF6E000EB06EAC94B896948E68
:10093000948CAB88AC8A120000EE60F0420EEE6A36
:10094000E806FDE135903592000EF86E000116EFD5
:0E09500003F02A6EA4A8FED72AC073FF12007F
:020000040020DA
:08000000FFFFFFFFFFFFFFFF00
:020000040030CA
:0E000000FF381F3CFFBF85FF0FC00FE00F4011
:00000001FF
